:020000040010EA
:2000000018F09FE518F09FE518F09FE518F09FE518F09FE50000000014F09FE514F09FE514
:2000200090010000D0020000D4020000D8020000DC020000E0020000E4020000F8B5020058
:20004000002528000E4D2B00002912D0040015782800521C604008263500002D07D006008E
:2000600040083700FF0700D558406D1EF5E7491EEAE70004000C01B00499F0BC01B00847E5
:2000800008840000F8B514480400002005000020060000200500202D05DA30002668064324
:2000A000241D6D1CF7E7002E01D100200FE00B490948FFF7C3FF0700094800880004000C3C
:2000C0003F043F0CB84201D0002000E0012001B00499F0BC01B00847008E1000FE6D0000A3
:2000E000FEFB100001607047016170474163704780B500231A00824208D200231900054BCF
:20010000994201D2491CFAE7521CF4E7019802B00047C046B80B000038B581204003050071
:2001200000200400102C04DA200002F2B9F8641CF8E7FFF7A7FF00281CD002F285F802F248
:2001400097F801210F48FFF7CDFF04210D48FFF7CBFF0D488021490501600C4880214905B3
:200160000160802149050848FFF7C0FFFA208000FFF7BEFF00F0BAF8002001B0029930BCE3
:2001800001B0084700FCFFFF00F4FFFF10F4FFFF00000FE11F00C0E3120080E300F021E158
:2001A0002CD09FE507D0CDE31F00C0E3110080E300F021E11CD09FE507D0CDE31F00C0E357
:2001C0001F0080E300F021E10CD09FE507D0CDE3230000EA002120000022200000202000F4
:2001E00024009FE510402DE920409FE5020000EA041090E40FE0A0E111FF2FE1040050E1D4
:20020000FAFFFF1A1040BDE81EFF2FE1880200009C020000050000EA041090E4042090E473
:2002200004C091E4043053E204C082E4FBFFFF1A043090E4000053E3F6FFFF1A1EFF2FE1C6
:2002400000C09FE51CFF2FE1E902000000C09FE51CFF2FE11901000000C09FE51CFF2FE14C
:20026000C50200000100A0E3F4FFFFEB000050E3DAFFFF1B0000A0E3F3FFFFEBF5FFFFEBF3
:20028000050000EBFDFFFFEA14020000D8000000F0020000002220000000000008109FE5CB
:2002A0001800A0E3563412EFFBFFFFEA260002007847C0460070A0E10700A0E1F6FFFFEBF0
:2002C000FDFFFFEA80B5FFF7F3FF019802B00047FEFFFFEAFEFFFFEAFEFFFFEAFEFFFFEAF2
:2002E000FEFFFFEAFEFFFFEA012070472847000038B50C03240B220020242300002B05D037
:2003000004681460001D121D5B1EF7E74C00084D2540084C2C439B25ED432C609724E44333
:200320002468E407FAD501B0029830BC01B0004700FF03000100005A10B500200400DC2006
:20034000C001844208DA8120400321180F482018FFF7CEFF8034F2E7019810BC01B00047DB
:2003600010B5A0B000200400202C06DA04206043694600220A50641CF6E704496846FFF7D8
:20038000B7FF20B0019810BC01B00047008E100080B50007000F9721C94309680122824077
:2003A00012040A40002A05D00102064A0A439B21C9430A609721C9430968C907FAD501989F
:2003C00002B000470400005A000000000000000000000000000000000000000000000000C6
:2003E0000000000000000000000000000000000000000000000000000000000000000000FD
:200400000000000000000000000000000000000000000000000000000000000000000000DC
:200420000000000000000000000000000000000000000000000000000000000000000000BC
:2004400000000000000000000000000000000000000000000000000000000000000000009C
:20200000741300EAFEFFFFEAFEFFFFEAFEFFFFEAFEFFFFEAFFFFFFFF00F09FE520FF1FE524
:20202000D4392000FFFFFFFFFFFFFFFFFFFFFFFFFFFFFFFFFFFFFFFFFFFFFFFFFFFFFFFF8F
:20204000000000000000000000000000000000004A2D4C696E6B2041524D20563720636FDC
:202060006D70696C6564204E6F7620323020323030382031333A30393A313800436F7079C1
:20208000726967687420323030332D32303038205345474745523A207777772E73656767D6
:2020A00065722E636F6D0000000000000000000000000000000000000000000000000000DC
:2020C00070B50C4C0C4E82B02500241D03E005F0B5FB0C350C34B54208D2616820682A68D4
:2020E0008142F4D1002105F0B5FBF2E702B070BC01BC0047488310007883100001C08FE2BF
:202100001CFF2FE1044C054D054E064FAE462047002809D0BE463047956910001121100023
:20212000C120100029211000044C054D0020AE462047044C044DAE4620470000A177100013
:2021400033211000097810006D781000F5B504000D00724800684107490F00916E49C00808
:202160000A68161848684010371808200099411A019805F0F1FA010022002B0000980028CD
:2021800013D03400761C2578AC4605001800A8406546284320707C1C3D78AC46009D100070
:2021A000A84065462843387003E03570761C3C707C1C0198884203D00B4133700A41227019
:2021C000564856490968019A89180160FCBD000070B5524C2068C01DC6084F4D28683200A7
:2021E000696849104118801905F0D6FA70002968091829606968081A68600020206070BDCB
:202200004548006870470000F1B504000D0016004248006800900AE037003A002906090E22
:202220002006000EFFF792FFF61B240A2D0A012E03DB092EF0DB0827EFE70098F8BD00000C
:2022400010B5040005E00822FF210020FFF7DCFF083C082CF7DA012C06DB012201210020D9
:20226000FFF7D2FF641EF6E710BD0000004850E0D002200000B523488168002901D0491E97
:20228000816000BDF0B5070003F0CEFA002827D11C4C052F01D2A060F0BD01256426A06845
:2022A000002807D0A6606068002819D003F0C0FA2570F0BD802F13D303F080FC0100012922
:2022C0000EDB084805F0E0FA08000749884204D36060257003F0ACFA01E000206060A66048
:2022E000F0BDC04600A3E11141420F0010B5054C2078002804D0002003F09AFA0020207003
:2023000010BD0000C8022000034A10605160C0460248002101607047D4022000F8292000D8
:202320000023C36042610160891841608918816070470000F0B504000F00E5687E68606924
:20234000C0007119884201D202F0E6FB3F6833003A00E168206801F1ABFC3300F01DC0083D
:202360003A18E168A06801F1A3FCE0688019E0602800F0BD00B5C168C91D0722914380688A
:2023800003F0ECF800BD000000B5C168C91DCB080021C16042688168006803F0CFFA00BD5C
:2023A00030B50400E068C01DC5080020E060E900A06803F0D3F82B006268A168206803F0BA
:2023C000BDFA002801D103F01BFA30BDF0B50400174805686435964E310094312000FFF759
:2023E000A9FFB18B47182000FFF7DAFF00281DD1F80861680A1810787B075B0F06D0D84048
:20240000010050780822D21A9040084319210140092901D10020F0BDC00601D50320F0BD0A
:2024200003480068281A0128D6DA0220F0BD0000C429200010B59EB0040003F0E1F90028E6
:2024400020D12069C108626851180A784007400F06D0C24013004A780821081A82401A43D7
:2024600019201040092801D100200BE0D00601D5032007E0202206A96846FFF751FF68467C
:20248000FFF7A4FF1EB010BD08604A60D21DD110490040187047000010B50400486800282D
:2024A00005D02000FFF746FF2000FFF779FF10BD00B513005A07520FDB080068C01801F1F2
:2024C000D1FB00BDF5B585B00C00002002900190574D019801210140182041436E183836F5
:2024E0000E2C01D2009401E00E200090069800680099884261D00198C00701D5002000E0CC
:202500000800069908602900B4313000FFF712FF0700012000998840401E40000490404923
:20252000401801F183FB298B7A1801003000FFF7BFFF28008430039001003000FFF7FAFE1A
:202540003849EA8A80180860012704E003993000FFF7F0FE7F1C00988742F7D32900BC31EE
:202560003000FFF7E7FE070004982F49401801F15DFB0100688B3A183000FFF799FF290066
:2025800094313000FFF7D6FEA98B401830613000FFF7F0FE00980E2812D1F068C01DC70896
:2025A0003A003168286D05F0F7F83A00B168A86D05F0F2F83069286602E01C480068F06063
:2025C000009B184802680599300000F11FFF05900298002807D0FFF72DFF002803D08035B9
:2025E0000E342C601AE01148F16801603000FFF7CBFE002801D08035F3E70098241A01981A
:20260000401C01900296002C00D062E73000FFF711FF002802D080350099296007B0F0BD85
:20262000000090E8F80320000000A0E8FC032000DC02200030B50C00C44D2A8829008C31C8
:20264000FFF722FF6A882900A431FFF71DFFAA882900AC31FFF718FFEA882900B431FFF7A6
:2026600013FF2A8929008431FFF70EFF6A892900BC31FFF709FFAA8929009431FFF704FF93
:20268000EA8929009C31FFF7FFFEAA8C2900C431FFF7FAFEEA8C2900CC31FFF7F5FE2A8D60
:2026A00029006831FFF7F0FE6A8D2900D431FFF7EBFE002C0AD06A8E29007031FFF7E4FED0
:2026C000AA8E78352900FFF7DFFE30BD00206867E86730BD70B501281FD09C4C002801D1E2
:2026E000242102E0022803D13221200003F060FE0A4D28001C3003F08DFDE08B03F054FDFA
:202700000600EE6101D102F007FAE18B300003F04FFE00213000FFF78DFF70BDB8032000E8
:20272000F5B50400204D002B33D1884E3100CC31FFF700FE070001200199884040001B4929
:20274000401801F173FA0100308E3A182000FFF7AFFE310068312000FFF7ECFDB18D40188F
:202760000090012705E0310068312000FFF7E2FD7F1C01988742F6D3D43631002000FFF7E6
:20278000D9FD2000FFF7F6FDE06828600098206101E02868E0602000FFF7F6FD002801D1BD
:2027A00003F02EF8FCBDC04600042000FEFF7FE8F5B50A00036900212C48007800284CD048
:2027C000019881424CD2D808009C646824185807400FA507ED0E4519032084432068002DA9
:2027E00006D0E84064682026751BAC40044320001C4C24681B19040AFF251B4E2840305C2F
:202800000706FF202040305C00043843240A2540755D2D020543200A305C28431060121D85
:20282000491CCDE7D808009C646820185C07640F8507ED0E64190325A8430568002C06D0A3
:20284000E5402E0045682020001B85403543054800681B181560121D491C01988142E1D3DF
:20286000FCBDC04648032000C8861000FC02200033B50400354D2900C43128003830FFF7A0
:2028800059FD154801F1D2F90100EA8D28003830FFF70EFE28003830FFF798FD002800D0AB
:2028A0003CBD00230222694628003830FFF738FF0028F5D10222694638352800FFF778FFA9
:2028C0000098C006C00E1F2801D004203CBD0198207000203CBDC0460120D0E433B504008E
:2028E0001A4D2900C43128003830FFF723FD164801F19CF90100EA8D28003830FFF7D8FDF5
:2029000028003830FFF762FD002800D03CBD00230222694628003830FFF702FF0028F5D176
:202920000222694638352800FFF742FF0098C006C00E1F2801D004203CBD019820700198D5
:20294000000A607000203CBDB220D0E0DC022000F1B591B00C0000250D2C01D2260000E0DA
:202960000D263C4F002D04D00D2E02D1012000902FE0002000903900C43138003830FFF756
:20298000D9FC0120B04080003149401801F14EF9FA8D010038003830FFF78AFD3900943123
:2029A00038003830FFF7C6FCB98B4018B86438003830FFF7DFFC786C019038003830FFF78B
:2029C000E3FC002841D138003830FFF733FD00283BD1009B721C03A938005030FFF7A0FEC3
:2029E000002832D11A2C14D30198786438003830FFF7CAFC002828D1721C03A9380050309B
:202A0000FFF7D6FE38373800FFF714FD00281CD105E0721C03A950373800FFF7C9FE0398F3
:202A2000C006C00E1F2801D004200EE0B7003A0003A9091D119804F0AFFE1198C0191190A8
:202A4000A41B6D1C002C87D1002012B0F0BDC046FCFFAFE8DC022000FCB5C04CA5440500DA
:202A60000C00002004900A9005908026760032000BA9BB48FFF754FC3200C02080000BA9D6
:202A80000918B848FFF74CFC09942000FFF7FAFB052C05D2B449B248FFF7FEFC070041D127
:202AA000B249AF48FFF746FCB1480190007C002804D0280001F1BAF8010000E0290001987B
:202AC0000288A748FFF7F4FCA548FFF769FC070028D1A8480890E80726D500200290012109
:202AE00002A8A54A6A441268126800F0A3FF641E0198007C002803D0029801F197F80290CA
:202B000008999748FFF716FC01994988421802999348FFF7CDFC9248FFF758FC070002D036
:202B200001200490FDE06D1C9448079002210D4230D0022C2ED30020009068468E4A6A4482
:202B40001268126800F076FFA41E0198407C002805D000980004000C04F0C8FD009001987E
:202B6000007C002803D0009801F160F8009007997B48FFF7DFFB01998988421800997848DB
:202B8000FFF796FC7648FFF721FC070001D00220C7E7AD1C042C52D303F0F6FA02003821D8
:202BA00004F06AFE101A069003F0FEFA0590A00880000699884201D2039000E00391039972
:202BC00005986D4A6A441268526800F033FF00200090694868440068806804F013FE03999F
:202BE000091A03229143009A8E1A002806D0382EEFD33000382104F03FFE361A002F10D137
:202C00000AAAB108009880088000059B1818FFF759FC0700AD19002F03D00198006F800035
:202C20002D1A00988019009003998842D1D1641A042CBCD2002F02D00420049071E002211B
:202C40000C422DD00020009068464B4A6A441268126800F0EFFEA41E0198407C002805D0A3
:202C600000980004000C04F041FD00900198007C002803D0009800F1D9FF009007993848C9
:202C8000FFF758FB01998988421800993448FFF70FFC3348FFF79AFB070000D077E7AD1CCC
:202CA000002C23D00020009001216846324A6A441268126800F0BEFE641E0198007C0028EC
:202CC00003D0009800F1B2FF009008992448FFF731FB01994988421800992148FFF7E8FB88
:202CE0001F48FFF773FB070000D019E724491C48FFF720FB1A48FFF753FB070011D1099820
:202D000005280ED21F491648FFF7C6FB070008E0012102A8184A6A441268126800F08AFEF2
:202D2000641E002CF4D1C620C00068440068390007800AD0C620C000684400684560C62087
:202D4000C0006844006804994180059803F050FAFFF7CCFA38000C498D44F0BDD4F9FFFFD5
:202D6000140320002C0320004C03200068032000EC022000800320002C0600008803200045
:202D800078032000540320003406000010B585B00121684603F00CFB68460078FFF79AFC71
:202DA000042101A803F004FB042102A803F000FB03AB0B4A02990198FFF74EFE03AC2088C6
:202DC0000006000E03F0CCFA2088002805D0049803F0D0FA608803F0CDFA05B010BDC046FE
:202DE00064861000FFB5944CA5440024019400940594944D80267600320007A92800383007
:202E0000FFF78EFA3200C020800007A9091828005030FFF785FAC420C0006844006802906A
:202E2000C420C00068440068FFF72CFA03F0ACF9049003F0B9F9069029008C3128003830E1
:202E4000FFF778FA2020285C002805D07B486844006800F1EBFE02E07848684400682A8A2E
:202E6000010028003830FFF723FB38352800FFF797FA0090069D02980499884201D20390F7
:202E800000E00391039E009800280CD16B4868440068C00713D501200190761E2800FFF7A6
:202EA000E7FC0090002872D16D1C644868440068401C02B4C421C9006944086002BC6048B0
:202EC0006844006840004BD45C48684400680221084214D0022E12D30191B61E2800FFF7DD
:202EE000FDFC0090002852D1AD1C544868440068801C02B4C421C9006944086002BC50481A
:202F000068440068000029D4042E27D3B70804200190B800361A39002800FFF719FD0090FB
:202F2000002834D1B8002D18444868440068B90040180DE002200190B61E2800FFF7CEFC5A
:202F40000090002823D1AD1C3C4868440068801C02B4C421C9006944086002BC022EE9D2A6
:202F6000002E14D001200190761E2800FFF780FC009000280BD16D1C304868440068401C5A
:202F800002B4C421C9006944086002BCE8E7002C26D101216846C822D2006A4412681268DA
:202FA00000F048FD00980590002819D0C420C00068440068412816D3042120486844C82271
:202FC000D2006A441268126800F034FD042101A8C822D2006A441268126800F02BFD22E016
:202FE0000598002805D0C420C00068440068412808D203990698C522D2006A4412681268A7
:2030000000F018FD02980399401A0290641C002800D02FE70098002805D0C420C000684416
:2030200000684128C8D3069803F0E2F8FFF75EF9059805498D44F0BDE4F9FFFF1C06000006
:2030400024060000DC0220002C06000007B5012101A803F0ADF968460079FFF73BFB04217E
:2030600002A803F0A5F90421684603F0A1F9009A1002000A0090034B08B401000398FFF7D3
:20308000B1FE0FBD70861000F1B504000D007948C67D007D401B871B042200210320FFF71A
:2030A000B3F8002F02D03800FFF7CAF853480068009008E000203A0021780006000EFFF7FC
:2030C000A3F8641CED1B012D0CDB082D01DA2F0000E00827002EEDD1092DEBDA0120691EDB
:2030E0008840E8E7002E09D0022E02DB701EFFF7A7F8012201210800FFF786F83AE0000027
:20310000F1B504000D005B48867D407D401E871B032200210120FFF777F8002F04D03A008C
:2031200000210020FFF770F834480068009008E000203A0021780006000EFFF765F8641CBA
:20314000ED1B012D0CDB082D01DA2F0000E00827002EEDD1092DEBDA0120691E8840E8E7DE
:20316000002E06D0320000210120761EB040FFF74BF8C046012200210120FFF745F80098E4
:20318000F8BD000031B51C480078012827D101240420051B684600780121A940491E014055
:2031A00001202041814217D1042200210320FFF72BF822006846017829410906090E012065
:2031C000641EA0400006000EFFF71EF8012200210120FFF719F838BD641C052CD8DB074859
:2031E0000068002803D101220021FFF70DF804216846FFF749FF38BDCD032000F8292000F5
:2032000010B5040004E0012200210020FEF7FCFF2000441E0028F6D110BD000071B5050044
:20322000144E307E002801D0052400E004240220FFF7A8FF0120611E884021000095727D88
:20324000012A12D14A1E00E0521E002A0DD08B1A0400DC40009B012595406D1E1D40AC4270
:20326000F2D1891A1800D04000906846FFF748FF78BD0000B803200033B504000D0000F14B
:20328000D5FC400005436846057029124170291481702916C1700121214001712121FFF7FB
:2032A0002FFF0400012200210020FEF7ADFF20003CBD000013B50C0000F1B8FC6946C200D4
:2032C00022430A7042094A70420B8A70420DCA70400F087123216846FFF712FF0400012252
:2032E00000210020FEF790FF20001CBD00B53A490978002902D1FFF7BFFF00BD0021FFF7D3
:20330000D9FF00BD70B505002A4C33480078002809D1022601212000FFF7AEFF2800FFF758
:20332000E5FF050008E004262800FFF7DFFF050004212000FFF7BEFF0420FFF723FF30002D
:20334000FFF75EFF280070BD17B523490978002902D1FFF7CBFF1EBD6C462070010A617057
:20336000010CA170000EE070124800F15FFCC100217141096171410BA171410DE171400F6F
:20338000207243216846FFF7BBFE0400012200210020FEF739FF20001EBD000010B5040081
:2033A000012C05DB0348FFF7A1FF601EFFF728FF10BD00000000A0E100B5000305494018D8
:2033C000FFF794FF04480078002802D00220FFF7E5FF00BD00000FE1D003200013B50C0036
:2033E000694600220A604A60087006216846FFF787FE6846002101702100FFF781FE1CBD71
:2034000003B56A4611606946202202430A7126216846FFF775FE0120FFF7F2FE00200CBDD4
:2034200000B5012002E0000000B50220FFF7F6FE0C20FFF7A7FE00BD00B50349096801809C
:20344000FEF7C6FE00BD0000F8292000F3B50500D64E707D0190307E002802D10124009404
:2034600002E0002403200090012200210020FEF7CBFEFFF7D5FF0020FFF79EFF9548FFF721
:2034800035FF9548FFF732FF307E002802D00420FFF784FF9148FFF729FF0220FFF77EFF23
:2034A0000020FFF751FF0700307E002802D10120FFF7A6FE381928820F20FFF763FE280092
:2034C000FFF7BAFFFFF7ACFF8548FFF70FFF0220FFF764FF0020FFF737FF001968820120E0
:2034E000FFF78EFE824F3800FFF700FF7D48FFF709FFA81CFFF7A0FFFFF792FF7848FFF7F3
:20350000F5FE0220FFF74AFF0020FFF71DFF0019A8820120FFF774FE3800FFF7E7FE72488C
:20352000FFF7F0FE281DFFF787FFFFF779FF0020FFF7DCFE0099401828836C480199012974
:20354000317E12D0002905D1FFF7D0FE0120FFF757FE02E00220FFF721FFA81DFFF76CFF6B
:203560000020FFF7F1FE001918E0002905D1FFF7BDFE0120FFF744FE01E0FFF7B7FEA81DDB
:20358000FFF75AFF307E002803D1FFF7DDFE001904E00020FFF7AAFE00994018E882280023
:2035A0000830FFF749FF307E002806D10120FFF727FE0120FFF724FE02E00520FFF7EEFE8A
:2035C0000020FFF79FFE00994018688328000A30FFF732FF012200210020FEF715FE022045
:2035E000FFF71CFE0C20FFF7CDFD05210120FFF7F5FEA88328000C30FFF71EFF0F20FFF7D8
:20360000C1FD28000E30FFF717FFFFF709FF3800FFF76CFE0020FFF775FE00994018E885FD
:2036200028002430FFF708FFFFF7FAFE0120FFF7C3FE0020FFF75AFE00994018288602201C
:20364000FFF7ACFE28002630FFF7F6FE307E002802D10020C04300E03800FFF747FE00192A
:20366000A88528002830FFF7E7FE0F20FFF78AFD2A352800FFF7E0FEFFF7D6FE0021C943C4
:203680000B20FFF7BDFE00210920FFF7B9FE00210820FFF7B5FEF7210D20FFF7B1FE8021DA
:2036A00049000C20FFF7ACFE0F20FFF76BFD324C20003230FFF7C0FEFFF7B6FE00210C20BD
:2036C000FFF79EFE0F20FFF75DFD34342000FFF7B3FEFCBDDF0080E300F02FE101009EE828
:2036E000020090E80110C0E4B210C0E0FFFFFFEA0000A0E1F0B507000D001E4E2B4CB0780D
:20370000A84207D1082239002000143004F082F800282ED0082239002000143004F03CF89D
:2037200020001C3002F076FD80273F01380002F03BFDE0613900FEF7E7FD0020217E002934
:2037400001D1012100E000213170002D00D03078B070607E70700848FFF778FEFEF750FD52
:20376000E269811A100002F04BFD0121E069FEF761FFF0BDFC022000DC02200003B50821AF
:20378000684602F015FE00216846FFF7B3FF0CBD10B5064C082200212000143004F05AF82A
:2037A0001C34200002F036FD10BD0000B803200000B5FFF7EDFF07E000B5FFF7E9FF0BE0D0
:2037C00000B5FFF7DBFFC046FFF7E0FA00BD000000B5FFF7D3FFC046FFF738FC00BD000067
:2037E000F0B5FFB0EBB0904C08222100143108A803F0D2FF08212000143002F0D9FD022182
:20380000684602F0D5FD022100A8801C02F0D0FD022102A802F0CCFD022102A8801C02F02D
:20382000C7FD68460588802189000AA8FEF76CFD607EE072012200210020FEF7E5FCFFF7EF
:20384000F3FD2000FFF7F8FD06210420FFF7C6FDE081A01CFFF7F0FD20210520FFF7BEFD52
:203860002082201DFFF7E8FD0F20FFF78BFCA01DFFF7E2FD2288210020310AA8FEF704FE8B
:20388000628821002831FEF7FFFDA28821003031FEF7FAFDE28821003831FEF7F5FD634EAF
:2038A00040228AA930003830FEF73AFD40228AA9C03130005030FEF733FD6846008880009E
:2038C00002F072FC0190002800D194E02100203130003830FEF72EFD30003830FEF760FD76
:2038E000019803905248006869460989401804902100283130003830FEF71CFD30003830B5
:20390000FEF738FD706C05902100303130005030FEF710FD30005030FEF72CFDF06D069017
:2039200055E0079842490968401A64D4049840490968401A5FD40598706430003830FEF704
:2039400023FD002801D101F05BFF002853D1E189C808F26B10184907490F03220240D20016
:203960008918B8430268002906D0CA40130042682020401A82401A439007D2D50698F06591
:2039800030005030FEF700FD002801D101F038FF002830D1218AC808726D10184907490F10
:2039A0000740FA008918032290430268002906D0CA40130042682020401A82401A430398A9
:2039C00002600398001D03906D1E2D042D0C280007D01748006869464988401807900327E6
:2039E000A4E72100383130003830FEF7A3FC38363000FEF7D5FC68460088451B280002F072
:203A0000B9FCA900019802F083FC0198002801D002F0EEFB082208A91434200003F0BCFEE1
:203A20007FB06BB0F0BDC046B8032000DC022000C42920001047000000B51E21002003F045
:203A400017FA02F0DBFA00BDF0B504000D00002605E0022F12D13000761C64280ED02900A7
:203A6000200003F005FA03F0CDF90700012F01D10020F0BDFFF7E0FF042FEAD10020C043BF
:203A8000F0BD0000F3B503F0C3F9040002F028FB0500002606E03000761C64281AD0009828
:203AA00003F0B6F9280002F01FFB200003F0AAF90700012F0AD1032003F0AAF9C41C2000AF
:203AC00003F09CF9019908600020FCBDFFF7B4FF022FE0D00020C043FCBD000070B50400F4
:203AE0000D00FFF7A9FF00210220FFF7ADFF0600064929430420FFF7A7FF05003543210017
:203B00000520FFF7A1FF284370BDC0461000002330B50C000025ED430221FFF7DFFF0028B4
:203B200001D0280030BD21000720FFF7ABFF002800D0280030BD000010B50C000221FFF7C0
:203B4000CDFF002802D00020C04310BD21000720FFF77AFF002801D00120C04310BD00000E
:203B6000FAB584B0040015005910FFF7B7FF002803D00020C04306B0F0BD072003F048F958
:203B8000060002F0ADFA0390049801900020009002900EE0FFF750FF022FEAD10299481C66
:203BA00002906429E5D0072003F032F90098002842D1039802F098FA0098002834D0300006
:203BC00003F020F9042802D1FFF736FFD1E7F01C03F014F90599012904D0022908D004291F
:203BE0000FD016E0A107C90EC84028706D1C10E002222240D100C8402870000A6870AD1CB6
:203C000007E02870010A6970010CA970000EE8702D1D059824180198401E019001D104989C
:203C2000A9E7002002900090300003F0EBF80700012FAFD10120009001980128B9D10320D5
:203C400003F0E6F80600BAE7FCB505000E00002407E03800019988402D18009908180090F5
:203C6000F61B002E14D0E84307053F0D0198C7407F1CBE4200D2370001238340009A3900A0
:203C80002800FFF76DFF002803D42418B842E0D02000FCBDF2B5060017001D000C00C00728
:203CA0000FD5002C0DD000232A0001213000FFF7CBFF002800D5F8BD241A012846D16D1CFF
:203CC000761C780037D4B0070FD5022C0DD301232A0001213000FFF7B7FF0028EBD44100B2
:203CE000641A012832D1AD1CB61C380011D4042C0FD3A70802232A0039003000FFF7A4FF50
:203D00000028D8D48100641AB8421FD1B8002D183618022C0FD3670801232A003900300065
:203D2000FFF792FF0028C6D44100641AB8420DD178002D183618002C08D000232A00210026
:203D40003000FFF781FF0028B5D4241ABEE00000F3B5040015001E007110FFF7BFFE0028F5
:203D600000D0B7E6019F2978022E0CDB0A00687801021143032E06DB0800A9780A04E97893
:203D80000906114301430422921B2240D0008140A419AD190720FFF757FE002811D17F1E1A
:203DA000E1D1684607490A780270401C0021017000AA521C6946082002F058F902F01EF936
:203DC0000198FCBDC8871000FCB505000E00002407E03800019988402D180099081800903B
:203DE000F61B002E14D0E84307053F0D0198C7407F1CBE4200D2370001238340009A39001F
:203E00002800FFF7A5FF002803D42418B842E0D02000FCBDF2B5060017001D000C00C0076E
:203E20000FD5002C0DD000232A0001213000FFF7CBFF002800D5F8BD241A012846D16D1C7D
:203E4000761C780037D4B0070FD5022C0DD301232A0001213000FFF7B7FF0028EBD4410030
:203E6000641A012832D1AD1CB61C380011D4042C0FD3A70802232A0039003000FFF7A4FFCE
:203E80000028D8D48100641AB8421FD1B8002D183618022C0FD3670801232A0039003000E4
:203EA000FFF792FF0028C6D44100641AB8420DD178002D183618002C08D000232A002100A5
:203EC0003000FFF781FF0028B5D4241A0098001BF8BD0000F0B505000E0017000221934818
:203EE000FFF7FCFD040010210220FFF7ADFD2043040029780520FFF7A7FD010021430C00A4
:203F000031000620FFF7BEFD20436D1C361D7F1EEED1F0BDF0B505000E0017000221834894
:203F2000FFF7DCFD040010210220FFF78DFD2043040031680620FFF787FD010021430C00CA
:203F400028788021490201430520FFF77DFD20436D1C361D7F1EEBD1F0BD000011B5734C32
:203F600069462000FFF7D4FD002810D10098000307D56F492000FFF7DFFD69462000FFF7BC
:203F8000C7FD0098800301D5012018BD002018BD00B567496548FFF7CFFD002801D1FFF7BD
:203FA000DDFF00BD10B5614C002805D005492000FFF7C2FD044900E004492000FFF7BCFD8D
:203FC000002010BD0B005FA009005FA001005FA030B50024E443554D0A492800FFF7ACFDF6
:203FE000002805D108492800FFF7A6FD002801D0200030BDFFF7B2FF04004D492800FFF74C
:204000009BFDF5E70F005FA00D005FA0F1B501214848FFF791FD17491748FFF78DFD424C69
:204020002568FA358026B604404F69463800FFF76FFD0098304002D02568FA3508E0206886
:20404000281AF2D50020C043F8BD2068281AF9D469463800FFF75CFD00983040F5D10021C3
:204060003448FFF769FD32493800FFF765FDFFF775FFF8BD0100FA050CED00E0F3B581B08C
:204080000026294C294D00E0012629492800FFF753FD01212748FFF74FFDFFF7CDFC012075
:2040A00002F08AFB01F00EF9019802F085FB01F00DF90298002800D1642002F07DFB206886
:2040C00016494718FFF74AFF012802D02068381AF8D517492800FFF72FFD002E07D0002171
:2040E0000F48FFF729FDB1210E48FFF725FD00211048FFF721FD002E0AD169462800FFF7AA
:2041000007FD00980003BFD4FFF728FF0028BBD002990198FFF77AFFFEBDC046DC05000058
:204120000000044004000440C4292000F0ED00E003005FA0FCED00E030B503000C00150055
:204140000020C043002B04D0012B0DD0022B10D030BD29002000FFF759FF01280DD0290074
:204160002000FFF78BFF30BD29002000FFF74EFF30BD29002000FFF781FF30BDFFB50024B5
:20418000E443042102A802F013F90421684602F00FF9009803900002000A009005008020F2
:2041A000C000854201D2019500E00190019801F0FBFF06001BD0002D17D00198854201D2E2
:2041C0002F0000E007003300039A39000298FFF761FD04000DD40298001902902D1B21003F
:2041E000300002F095F8BC42E5D00098441B002D03D02900002002F08BF8002E02D0300078
:2042000001F0F6FF200004B0F0BD0000FFB50025ED43042102A802F0CBF80421684602F0E5
:20422000C7F8009803900002000A009004008020C000844201D2019400E00190019801F06B
:20424000B3FF060010D1002C03D02100002002F0AFF8002E02D0300001F0CAFF280004B026
:20426000F0BD029840190290002C17D00198844201D2270000E00700E41B3900300002F05F
:2042800097F83300039A39000298FFF7C3FD0500D9D4BD42E5D00025ED43D4E7009DDAE762
:2042A00030B5A9B0002404E021A8694609780155641C0121684602F07BF868460078FF2867
:2042C000F2D1220001A921A8FFF704FE0500A10001A802F01DF8280029B030BD10B5AAB02B
:2042E00000240CE0042101A802F062F822A8694609780155A00002A9019A0A50641C012162
:20430000684602F055F868460078FF28EAD1220002A922A8FFF7FEFD2AB010BD0FB5002095
:20432000019014210291039004E06846017801A802F03EF80121684602F03AF8684600789B
:20434000002806D1039A02990198FFF7F5FE04B000BD012100A8401C02F02AF86846407893
:204360000128E2D0022802D0032804D007E06846017802A8DCE76846017803A8D8E76846AD
:2043800001780020D4E7000030B591B00400022100A8801C02F00CF86846418801A802F030
:2043A00007F88020C00001F0A5FE642C10D0652C11D06E2C12D06F2C13D0792C14D07A2CFF
:2043C0001BD07B2C1CD07C2C1DD0822C1ED020E0FFF7D4FE1CE0FFF719FF19E0FFF760FF0E
:2043E00016E0FFF77BFF13E00121684601F0E0FF68460078FFF7D6FD0AE0FFF7E9FD07E028
:20440000FFF7C6FD04E0FFF7A9FD01E0FFF786FF050001F083FE280001F0ACFF11B030BD1E
:2044200010B504000E480078FF2809D105220D490D4803F0EFF9002804D000F04FFF10BD30
:204440000028FAD0002C01D000F03CFF00F042FF002CF4D0142002F0AFF900F037FF10BD60
:2044600004FD10000086100010FF1000F1B585B000240025022104A801F09AFF6846008AC1
:20448000C01DC01000900321484301F08DFE01900098019908180290009802990818039059
:2044A000019800280BD100984100002001F080FF0099200001F02CFF009E062550E000998F
:2044C000029801F075FF0099019801F0A3FF01F0A7FF0099091A0E1B002803D0FF2EF6DDA1
:2044E0003F208643F7000098814206D16846008AC01D4007400FC01F3F182D062D0E1FD12C
:204500002048007800280FD139000298001901F025F83B0003980219029801190198001962
:2045200001F066FA050012E0012810D13B0003980219029801190198001901F05BFBF1E7B3
:20454000FF1DFA1000210398001903F083F931000398001901F012FFA41900988442B6D168
:204560006846007DCF2804D0B00606D101F00AFF03E02806000E01F0F3FE019801F038FEFD
:2045800006B0F0BD09342000F0B588B00221684601F00EFF022103A801F00AFF022104A818
:2045A00001F006FF022105A801F002FF022106A801F0FEFE6846008803214843093001F076
:2045C000F3FD040068460088211801910D1868460188200001F0ECFE68460188019801F0CE
:2045E000E7FE68460699418005998183039F008804990904090C6E18C000029002992000AA
:2046000000F0ACFF01F01AFF00F058FE00F05EFE3800471E000410D0029B2A002100019861
:2046200001F0E6F930787178090201436846808B0840694649888842EAD101F065FF6846C1
:204640000188280001F064FE200001F0D1FD08B0F0BD0000F3B581B014006846808C25182E
:20466000DE003100029800F079FF012002F0A4F800F024FE00F02AFE0D4F38686946098C10
:2046800040180090330022000299019801F0B0F928786978090201436846008D084069460D
:2046A000898D884203D000983968401AEAD5FEBDC429200070B585B00221684601F078FE9B
:2046C000022101A801F074FE022102A801F070FE022103A801F06CFE022104A801F068FE30
:2046E0006846008803214843093001F05DFD04006846008825182E1868460188200001F04C
:2047000057FE68460188280001F052FE049B039A029901980004000C0904090C1204120CCE
:204720001B041B0C0FB404A80388320021002800FFF790FF04A80188300001F0E9FD2000DD
:2047400001F056FD09B070BD70B5C0B0802464002100684601F02CFE21006A460B48030081
:2047600015781E782E40AE4207D1521C5B1C491EF6D12200694600F0B1FE0020FFF750FEF9
:20478000002001F0EDFD40B070BD000000FF100070B5A1B0002600240421684601F008FE68
:2047A0000BE0C00705D5300001F06AF901A94851641C761C009840080090A50000980028BF
:2047C000EFD1290001A801F0A3FD21B070BD000030B5A1B0002500240421684601F0E8FD90
:2047E00010E0C0070AD50020C043022D03D2A800094A1018406C01AA5050641C6D1C009841
:2048000040080090A10000980028EAD101A801F07FFD21B030BDC046040420003FB5684600
:2048200000211022121F8150FCD10A2400250F48019001F0C3F9002802D5012000900FE0CF
:204840002D180199884200D201900299814200D20290641EEDD128000A2103F00DF803916B
:204860001021684601F054FD3FBDC04600CA9A3B10B5C0B0802464002100684601F098FDE4
:2048800022006946024800F029FE40B010BD000000FD100000B501000020054B02019A5AFF
:2048A0008A4204D0401C0428F8D30020C04300BD0E04200000B5FFF7EDFF002804D401015A
:2048C000934A511800224A8100BD0000F0B5A5B0012100A8801C01F06BFD042103A801F06E
:2048E00067FD042104A801F063FD012100A8C01C01F05EFD012102A801F05AFD022168465B
:2049000001F056FD824C68468078642802D065283CD03FE06846008800280CD14020205AB4
:20492000401C402160526946088068460088FFF7B1FF0028F2D568460088FFF7ABFF754972
:20494000002804D4000120180968C16022E068466A46127A4272C078049A039B002502E071
:204960006D1C042D16D22E0127000A37BF5B002FF6D1A5192B606A6028726846407A6872FF
:204980006846008868810868E86003E068460088FFF790FF05A801906846018801A802F092
:2049A000E7FE042101A802F0E3FE102101A802F0DFFE042101A802F0DBFE00252E01A159E1
:2049C00001A802F0DDFE201D815901A802F0D8FE20000830815D01A802F0C4FE20000930ED
:2049E000815D01A802F0BEFE20000A30815B01A802F0BEFE20000C30815901A802F0C0FE66
:204A00006D1C042DDAD300F055FE010001A802F0B7FE4C2105A801F07BFC25B0F0BD000097
:204A200070B501F027F8324908680024012817DB304A904200D10020401C08602E498842D5
:204A400017D3FA21890002F017FF2C49884203D2002001F0D9F90CE0002001F0E3F908E008
:204A6000002806D5401E08602549884201D101F0A9F8274DE86C401CE8640A282DD1EC64E1
:204A800000F018FE1F498842686C29D31E4988422BDA002802D1A86C401CA864686C0A3053
:204AA0006864FDF7E7FB286D401C28650A2814D12C6518480668200129000A31095A00294F
:204AC00008D02818C168711A104A914202DB4089FFF7F0FE641C042CEDD301F079F970BD53
:204AE000002802D0A86C401CA8646C64D9E7C0467C2A2000FFFFFF7FF51A0000DE03000078
:204B0000F0D8FFFFD6060000005C26058813000004042000C429200000B501F08FFC00204B
:204B200001F08EF9F9E7000030B586B00500F42D02D1FEF73DFEB9E1F52D02D1FEF73CFE1B
:204B4000B4E1F72D02D1FEF73BFEAFE1F82D02D1FEF73EFEAAE1C22D02D1FFF739FEA5E1E2
:204B6000EB2D02D102F0C0F8A0E1FDF77FFBCE2D01D0CF2D09D1012001F008FC002803D1FD
:204B80002806000EFFF772FC90E1002480214900012D00D125E1022D00D115E1032D00D1FA
:204BA0000AE1042D00D12BE1052D00D1A6E0062D00D122E1072D00D1C0E0082D00D130E1B0
:204BC000092D00D16AE10A2D00D16AE10B2DDBD0C02D00D1E3E0C12D00D11FE1C72D00D148
:204BE00044E1C82D00D1E0E0C92D00D1BFE0CA2D00D1BFE0CB2D00D1BFE0CC2D00D1BFE06C
:204C0000CD2D39D0D02D00D1C0E0D12D00D1C0E0D42D00D1C0E0DC2D00D182E0DD2D00D12B
:204C2000CFE0DE2D00D1AEE0DF2D00D1D1E0E62D00D17CE0E72D00D17DE0E82D00D1EAE09B
:204C4000E92D1BD0EA2D35D0F02D6DD0F12D00D1F5E0F22D00D1BFE0F32D00D1BEE0F62DD8
:204C600000D100E1FA2D00D1EFE0FB2D00D1E9E0FE2D00D1ECE017E1CD2083E70121684612
:204C800001F096FB012100A8401C01F091FB022001F07CFB00280CD1684600780002694689
:204CA000497801438248814200D1824C200001F061FBFBE0012100A8401C01F079FB0121CE
:204CC000684601F075FB012100A8801C01F070FB012100A8C01C01F06BFB6846807800025E
:204CE0006946C97801437248814206D16846C378827801784078FFF747FBD7E0022102A85C
:204D000001F056FB684600896B49884201D16846048168460089FA218900484300F088FDBC
:204D2000C4E000F0CFFAC1E000F042FCBFE7654801F0EEFABAE0FFF707FDB7E003AC00F051
:204D4000B9FC208000F0D6FCA07000F0DBFCE07000F0DCFC207100F0C7FC607100F0E0FC6C
:204D6000A07100F0D9FCE071082103A8E0E700F02BFD9BE000F02AFD98E000F02DFD95E0C0
:204D800000F02CFD92E000F095FA8FE0FFF7FCFB8CE0FFF78FFC89E001F0F6F987E703A85E
:204DA00000F060FE062103A8C2E700F01FFD00F0A9FC01F0D5FA79E000F084FA022001F0EF
:204DC000FBFC00F083FA71E000F074FA022001F0F3FC00F073FA69E03B48A9E7FFF748FDCA
:204DE00064E001A800F068FB040001980004000C01F0BAFA019920009AE700F0E5FA55E0E2
:204E0000042001F0B1FA2D4801F0AEFA8020000101F0AAFA4AE00421294889E7FFF7B8FCB4
:204E200044E00121684601F0C3FA68460078002802D000F04FFA39E000F050FA36E000F01E
:204E400019FA33E000F018FA30E0FEF7C9FC2DE0042101A801F0ACFA042105A801F0A8FA89
:204E60000599019864E7FFF7D9FC1FE00121684601F09EFA0190002818D168460078FE289F
:204E800003D0FF2804D1032004E01048007801E000F0FCF90190042101A849E7FFF716FD0E
:204EA00004E001F007F801E0FFF736FE06B030BD01030000FE030000FFFF0000E32E00005C
:204EC0000886100000FF100000FD10000934200030B504001000020020785040641C0822EE
:204EE000012505404008002D00D05840521EF7D1491EF0D130BD0000004BE9E70884000076
:204F0000FCB589B007000E00129C159800251399C91DC908059116994907490F0791002CFE
:204F20003ED00091C108149A5118049101210722024091400906090E02911698C008109927
:204F40000818019013E000F05BFC04980078029908421ED1059B149A1199109800F0EEFC04
:204F6000002812D100F04CFC6D1C761E16D0009A39680198FEF076FE3F1D2300149A0A99E5
:204F8000099800F0DBFC0028DDD00020C0430BB0F0BD1798B6490968401AEED52800F6E708
:204FA0000695079800900698002803D1109804901A9802E0199804901B9802901898B04291
:204FC00001D2039000E003960398361A1698C008049908180190039C009A39680198FEF0E2
:204FE00041FE3F1D009813994018C108019A511801914007400F0090641EEDD10398189969
:20500000884201D2029800E000200090139C0398444311980290E01DC008059000980028A3
:205020001AD0059A029902F0B7FB6007400F019010D0E00800990C180821200000F08EFA1B
:205040002078FF21019A9140884320700821200000F084FA0098029000F0D2FB059B149AE5
:205060000299049800F06AFC00288ED1069801214140069103982D18002E92D100F0C0FB28
:205080008CE70000F1B577498D440024009401F07BF8099001F088F80B900DA801F0AEF958
:2050A0000EA801F0ABF903A801F0A8F90FA801F0A5F910A801F0A2F908A801F09FF904A8F9
:2050C00001F09CF90D98C01DC6080E98C01DC00802900398C01DC70802983018C0194500D6
:2050E000FF20801C854200D3B4E0290011A801F05FF908985E49096840180890700011A9CA
:2051000008180C9002980C9908180A9002980A9908180590C0190690012001900298002805
:2051200026D180200001039902F0A6FB01910498884200D20190019B039A0699FFA8483056
:2051400002F0DAFA019B039A059991A802F0D4FA01980499884205D28022520091A9D1A83B
:2051600002F01AFB91A80590FFA84830069003E0C1000A9800F0F2F901984743F9000698CA
:2051800000F0ECF911A88519F100280000F0E6F9330051AA290011A800F0D0FB00F030FB15
:2051A00004980790079885000998854200D3050029000B9801F02EF9002601F031F9291AF0
:2051C000032291438F1B002801D0402FF5D30098002821D4244B6B44FFAAFF324932D1A95A
:2051E00001980FB40C9B149A139955A80FB40B9B0A9A0E990D980FB4169B189AB9088C4643
:20520000B0108100179840186146FFF779FE0CB00090002800D42418F619AE42CDD1079872
:20522000A908401A0790BDD1104868440078002805D00098002800D40094042107E00498F5
:20524000844201D0012000E0002000900121684601F05EF80B9800F0CBFFE920C000854400
:20526000F0BDC046BCF8FFFF4406000044070000C4292000002005E701B50121684601F0A4
:2052800097F80120FFF7FEFE08BD000070B50400074D28780600012803D1012C01D001F098
:2052A00099FD200000F0B4FC2C70300070BDC0460934200000B500F039FA00BD00B500F002
:2052C00037FA00BD00B500F039FA00BD00B500F03BFA00BD00B500F04BFA00BD00B500F068
:2052E0003DFA00BD7047000030B50400064D00222900FFF701FE0004000C615B884201D11F
:20530000002030BD012030BDFE6D000000B5010000200A78202A07D1491C05E00A2358437B
:20532000101830380004000C0A78491C302A01D33A2AF3D300BD0000F0B58BB002A9204ADC
:205340002424241F13590B51FBD167300090001DFFF7DCFF01900098C01DFFF7D7FF040043
:2053600000980C30FFF7D2FF050000980F30FFF7CDFF0600002704E000201FE07F1C0C2FEE
:20538000FAD0032200990320784302AB181802F041FA0028F2D10B4820180C2148433F042C
:2053A0003F0CC0191F21484301990904090C40181821484340193C21484380190BB0F0BDE4
:2053C0000C86100030F8FFFFF0B5C2B0002000F0C7FF002000900221684600F0E9FF009827
:2053E000324988420BD3022101A800F0E1FF00988004800C69468988890301430091802481
:205400006400210002A800F0D3FF0098DC21C901884232D102A8FFF78FFF05008120400358
:20542000FFF78AFF002D03D0002801D0A84224D2204E3500220002A9280000F04FF86D27B1
:205440003619210002A800F0B3FF220002A9300000F044F87F1EF3D12800FFF745FF0400A0
:2054600002D0280000F058F8200000F079FF642001F0A2F900F0A6FB15E0009D802202A9EA
:205480005031154802F088F9260004E0210002A800F08EFF3619AE42F8DB054801F08CF994
:2054A000002000F05DFF42B0F0BDC04601800000DC050000008E100000B501000548064A88
:2054C0001378002B00D01000002901D070220A6000BDC04650201000FC292000F0B504000F
:2054E0000D00160009E0002000F08EFC7F1C70008742F8DB002000F095FC32002900200043
:20550000FEF05EF832002900200002F083F9002800D1F0BD0027EAE730B5C0B004008025C2
:205520006D002A00FF21684602F094F92A0069462000FFF7D3FF40B030BD0000004B18473F
:20554000C1352000982080024B490860A649802292010A609B4908607047000000B5C908E8
:20556000114A1268114B9A421AD30E4A04290FD30378D35C03704378D35C43708378D35CE6
:205580008370C378D35CC370001D091F0429EFD2002905D00378D35C0370401C491EF7E78C
:2055A00000BDC046C88610008404200070170000354800687047000030B5224800F038F98F
:2055C00004202C4908600021C9432B4A1160EC22D2022A4B1A602A4B1A60644A1160824A0C
:2055E000194B1360854A194B1360764A184B1360244A184B13604C4A13680224224A5D0A4A
:2056000028409D0B25400543580F012303402B439800114B185810601C4801600F48016040
:205620000F48982189020160FFF78CFF0D480E4901600E48FF2101600D4870210160144866
:20564000046030BD204E00000002108181610000810310010088002030861000A4F4FFFF7D
:20566000A0F4FFFF0480FDFF000B09031480FDFF1080FDFF10FCFFFF00F4FFFF70F4FFFF87
:2056800004F4FFFF64F4FFFF9804200060F4FFFF0080FDFF00B5002802D153480121016066
:2056A00000BD000000B5002802D154480121016000BD000000B502E0012001F07DF87B48C0
:2056C00041780029F8D0406A05494843054902F0DBF80800642800D200200004000C00BD37
:2056E000DC190000FF0300000F4800680104890E04E000000C480068410EC04601200840FA
:205700007047000008480068810EF7E7064800680104090FF2E7000003480068810DEDE7EC
:2057200001480068410DE9E73CF4FFFF2E4801E03248C04680214900016070472F4880217B
:2057400049030160284805E027488021490301602A48C0468021016070470000534800219D
:2057600001700248802109060160704714F4FFFF10B54E4C2078002822D1012001F01CF868
:20578000FA204000FDF0EAFF80200006164908600C490860012001F00FF800200021A17044
:2057A000A062A181E181218203004A00A21890808A00A2185061491C0329F6DB01202070A1
:2057C00010BD000010F4FFFF074801E00B48C0468021890101607047034801E00748C046AD
:2057E000802189020160704734F4FFFF8020C00151490860014908607047000030F4FFFF51
:2058000000B5974800687849884209D3054800680028FBD1754800688005FBD5FFF792FE7C
:20582000002000BD0441FDFF8D4800687047000030B504001D4AD4622ED001000123002588
:205840001648007801280DD11548814208D2154802F012F8891E116201291DDA136230BD7B
:20586000156230BD0F4802F007F80A3900D500211162B8208002844202D37D48112101E003
:205880001921094811630019401E210001F0F4FF0906080C0343536330BDC046093420001E
:2058A00080841E00808D5B0060E3160058042000FCB505000E001C00002780208002F10768
:2058C00001D51B4900E01C490860E80701D5184800E01948802189010160174849000160E6
:2058E0006D0876087F0813480068002801D0FDF037FFFFF70BFF002802D03800802707432C
:205900000B488021C90101600A480068002801D0FDF026FF641ED0D1009808216A469288F5
:20592000891ACF4007700448802189010160FCBD30F4FFFF7804200034F4FFFFF0B5040020
:205940000D0010001E009B494A6AE62A01DA0520F0BDC96A1F4A204BB827BF02B9420DD335
:20596000310003B429002000FDF07CFE1B4806601B4880214900016002B029E01A4FB942F9
:2059800011D3310003B429002000FDF06BFE02B01448297801606D1C144800688005FBD5EA
:2059A000761EF5D114E0002906D1F30002002900200000F0E7F9F0BD070008233A002178D9
:2059C0002878FFF775FF6D1C641C7F1C761EF4D10020F0BD0000FEFF0040FDFF0C01FEFFB0
:2059E0002001FEFF0C00FEFF701700001000FEFFF3B514001D0019480068E62801DA05203C
:205A0000FCBDEE0805D033000098FFF797FF070000E00027FFF7F4FE002F1DD16D076D0FA8
:205A20001AD0019880190190009880190090A4190B480068002807D12B0022000199009801
:205A400000F0A0F9070007E02B0022000098017801980078FFF72CFF3800FCBD7C042000AE
:205A600084042000024901600421818070470000006CDC02014859490160704740FDFFFF6D
:205A800000B54C4900280ED001280ED002280ED003280ED004280FD00A280FD00B280FD070
:205AA0000C280FD010E0087800BD887800BD0C2000E00E20085E00BD1020FBE7888800BDAD
:205AC000C88800BD088900BD0020C04300BD000070B53848C16B314A12688B18846B641CB3
:205AE00000220121082C04D1DB1043620024130041708463C36302240378002B4AD0836A01
:205B00005B1C8362264D2D68264E3668AD1B264E7543AD1285810E26865FAE4200DAC5812D
:205B2000642B04DB1023C35EAB4200DA05821F4B9D420EDB4269521C42618388934200D2B5
:205B40008280022A09D38170FFF7C8FBFFF7CAFB20E0426116498D420ADB8269521C8261E4
:205B6000C188914200D2C2800A2A06D38470EBE78261FF2192318D420BDBC269521CC261EB
:205B80000189914200D20281282A03D303218170DAE7C2610848046070BDC0464080FDFF8F
:205BA0004480FDFF4880FDFFC8190000B90B0000E9030000580420000080FDFF00B5FDF036
:205BC00039FE00BD00B500F039FC00F0BFFF024802490160FEE7C04600FDFFFF010000A5C7
:205BE00001489021A7E5C04614FCFFFF42489021A1E5000010B5040008000449096802B405
:205C0000210000F0C7F8002018BD00007804200070B51549154A164D1023164E114C0028C2
:205C200004D001280BD0022814D070BD34602B6088208002106098020860400910E0580104
:205C4000086014600C4804600C48046014600C48036070BD34602B6098208002106058017E
:205C6000106070BD1000000830F4FFFF34F4FFFF60F4FFFF14F4FFFF00F4FFFF10F4FFFFDB
:205C800064F4FFFF10B53A4C226063601A48402202602020194A1060194A10601D48042287
:205CA0000260C822520002600E480F4A02600F4A0F48C90001F0E0FD491C480810600D4812
:205CC0000021C94301602848216801602748616801600020274908602749086021480121E8
:205CE000016010BD0400FCFFC00808002000FCFF0080B6050C00FCFF10FCFFFF04F4FFFF4A
:205D000070F4FFFF034820210160164802210160704700000000FCFF134A1268026013480C
:205D2000006808607047000031B5040000F086FB0C48022101600C490B680C49A34201D2D4
:205D4000E21A09E00A4D2A68D31A6D685B190B6008490A600849A21A0A600121016000F02F
:205D600063FB38BD2001FCFF0001FCFF0401FCFF9C0420001001FCFF1401FCFF00487047DD
:205D80005086100008B4024B9C4608BC6047C0466837200008B4024B9C4608BC6047C046A6
:205DA000C438200000B50A214143414A51188A78002A01D0497800E00978002902D0FFF75F
:205DC00069FC00BDFFF76EFC00BD00007047000030B50024364DA888002810D0401EA88083
:205DE00000040CD16878002801D0298900E0E988012242406A70A9802000FFF7D3FF0A3D0F
:205E0000641EE8D530BD000000B50A214143284A511801220A708978002901D1FFF73AFC52
:205E200000BD000000B50A214143214A511800220A708978002901D1FFF734FC00BD0000F2
:205E400000B50A2141431A4A51180A78012353400B708978002901D1FFF7A4FF00BD00000B
:205E600070B5012823DA0A224243114B9A180B8893708B88D380CB881381CC880023012598
:205E8000002C02D1938055700BE08E88002E01D1938005E04E88002E01D09680F3E7948059
:205EA00053700988002900D19380FFF77BFF70BDA404200037B50221684600F079FA0024D8
:205EC0001BE0022100A8801C00F072FA022101A800F06EFA01AD0221A81C00F069FA0221D5
:205EE000281D00F065FA0221A81D00F061FA01A968464088FFF7B4FF641C68460088844296
:205F0000DFDB3EBDF3B584B03B488169CB104C07640F01940824019D641BA24201DA0092B3
:205F200000E000940124009DAC40641E056AEE180296466AF6180396019E002E17D0039E04
:205F400040B43678B44601AE377C2740029EB7406646374340BC3770029EB44636786F467F
:205F60003F7D3C40019FBC40344366460BE0039FBC466E46377C26003E4067463E70029E95
:205F80006F463F7D3C403470009C121B0919002A0CD05B1C446A6E46367C009F3E41E6549C
:205FA0006C46247D009E3441EC548918816106B0F0BD000010B5104CA169002919D0606A4E
:205FC0000C4A1278002A0AD107229143FFF7C6FAA369E269616A206AFFF70AFD07E0012A6E
:205FE00005D10B00E2690100206AFFF703FE0020A06110BD0934200040002000DAE7000087
:2060000010B50400FFF7D6FFE01017490968091808786207520F08D0D040030048780821EC
:20602000891A884018430006000E10BD10B50400FFF7C0FFE0100C490968091808784A7822
:2060400012020243887803041343C91C0878000618436207520F06D0D04003004878202110
:20606000891A8840184310BD5C002000F6B582B00400C01DC50830D02F4E7069B169C91D30
:20608000C910401A80218900884206D2FFF792FF7069B169C91DC910401A854201D200953F
:2060A00000E00090B0690190009E092C01D3082700E027003A000398017802980078FFF793
:2060C00021FF0298401C02900398401C0390E41B761EEAD100982D1ACED1019804B0F0BDC8
:2060E000034800687047000001490860704700005800200010B504000320604300F054F88A
:20610000002809D00C49C86102190A62620082184A624C6100228A6110BD000010B5064C33
:20612000E069002807D000F063F80020E061206260626061A06110BD4000200000B5002261
:206140004260016029490A68002A01D1086000BD0A0000E01A1D1368002B01D09842F9D2FA
:206160004360106008680028F1D000E0080041680029ECD0026883188B42F7D14B6843604D
:20618000096851180160F2E700B500201749096804E00A68904200D2100049680029F8D198
:2061A000002800D0083800BD10B501000020C91D0722914308310D4A00E01A1D1368002BD4
:2061C00013D01C68A14208D218005B1813600268521A1A6042685A6003E0EED118005B686C
:2061E0001360002801D00160083010BDB004200000B5002803D008380168FFF79FFF00BD4F
:20620000CA1D07218A430832083801680260891A801893E710B504002068FFF7E9FF002059
:20622000206010BD8AE7000010B502001423084C10000A2101F020FB3030E05410000A2138
:2062400001F01AFB0A009B1EF2D11620207010BD9800200011B52548FFF7EAFA2449254880
:20626000FFF7E0FF24480078012802D0022805D006E022480068FFF7D7FF08E02048F9E7B7
:2062800020480078042802D21F49401C087000F02FFE06E0FFF7D4FD322000F08DFAFFF759
:2062A000E9FB00F01FFE0028F4D00120FEF7B8F8FFF700FAFFF78AFD144C0020FFF7A4FDB7
:2062C00001202060FFF78CFC0121684600F070F8FFF78CFC0020C04320600020FFF7A2FDA1
:2062E00068460078FEF720FCE7E7C046204E000010250000B404200001FD100000FF1000FB
:2063000008FD100000FD10008E0020007C2A200070B588B005000C001FD0002D11D16846CD
:2063200000212022121F8150FCD1212C0ED320260DE026003100280001F030F8AD19A41BAD
:206340000BD02D488442F4D3461EF3E726003100684601F023F8A41BE7D108B070BD0000B5
:2063600001B5012102E0000001B50221684601F015F808BD01B50421F8E7000000B501F0B9
:206380002DF800BD00B501F005F800BD30B588B00400212C01D3202500E025002900684658
:2063A00000F006F8002801D1641BF2D108B030BD70B588B004000D0002D1002008B070BDC8
:2063C000002C08D113E02E003100200000F032FEA419AD1BF1D008488542F4D3461EF3E7C4
:2063E0002E003100684600F025FEAD1BE5D0212DF6D32026F5E700000108000011B50400F4
:206400000221684600F016FE684600882060002018BD000000B500F03BFE002000BD000041
:2064200000B500F059FE00BD7847C04600C00FE180C0CCE30CF021E11EFF2FE17847C0464F
:2064400000C00FE180C08CE30CF021E11EFF2FE17847C04613F021E31EFF2FE17847C046F4
:2064600093F021E31EFF2FE105480178491E01707047000002480178491C017070470000C3
:20648000C829200030B505000C00FFF7D7FF207E28432076617BF8220A40082A06D1617E62
:2064A000014203D0200000F045F830BD03480078002801D1FFF7B8FF30BDC046C92920001D
:2064C00070B50500FFF7BAFF0D4C6078401C60700C4E3068017E294205D145763068082158
:2064E000417300F02FF93068057E002101766078401E6070000601D1FFF796FF280070BD5F
:20650000C8292000D029200000B50148007831E1C929200010B5FFF791FFA54C2078401E85
:206520002070000605D186480078002801D000F049F911E170B581680024002906D00A68E9
:206540004968002A00D051600A608460417B8907890F4173964D14D177490A68002A16D1EE
:2065600008602878002807D101202870FFF75CFF00F028F92C7004E07148017802220A43D5
:2065800002706878002801D1FFF74EFF70BD137B067BB342E4D38242F3D1E2E730B504004A
:2065A000207B374900E011000A68002A02D0157BA842F8D322600C60607B002804D1FFF760
:2065C0003DFF2000FFF7B6FF30BD0000F0B5FFF735FF5B480178FE220A400270574C784D98
:2065E0002868FA21090140182060234E234F0EE03860016831600021017438688160FFF79E
:2066000013FF3868406801F0FDF8FFF717FF3068002806D081682A68891A0129E8DB8068A5
:206620002060FFF701FF1648066807E070692168411A00D52060FFF7F7FE3668002E1AD07E
:20664000FFF7FCFE3C480168002904D0317B0068007B81420FD3707B4007ECD570692968CF
:20666000401A0128E2DA3000FFF764FFFFF7E6FE707B0028DAD1F0BDD8292000DC292000C7
:20668000CC292000F0B54A4C00206070FFF7E6FE294D05E030682860FFF7DAFEFFF7DEFEC5
:2066A0002E68002E20D0777B38001DD0780711D5706943490968411A012906DA3000FFF749
:2066C00039FF707B002805D10EE01C490A68821A00D50860FB2038401028DBD1B068806884
:2066E0004068407B0028D5D115480178C90706D5FFF7AEFEFFF76AFFFFF7B0FEF4E70178EF
:20670000FD220A4002702B482968002909D02968497B0029296802D08968896849680160C3
:2067200006E0016000202070FFF792FE00F0ACF9F0BC01BC00470000D429200068002000F2
:206740000434200010B51A4C2078401C207000F039F82078401E20706078002801D1FFF7C3
:2067600063FE10BD00B500F031F81148012101704078C046002801D1FFF756FE00BD000072
:2067800010B504000A480078002806D0FFF74CFE0B480068001B09D5FAE7FFF74FFE054803
:2067A0000068446104214173FFF7CCFF10BD0000C8292000D0292000014909684018DFE762
:2067C000C4292000004B18472C681000004B18470C691000F2B5040015001E00069F1C226E
:2067E000002101F037F80B480178491C0170684600782073F0192C3803218843002101601F
:2068000005494162856260602000FFF7C7FEFFF781FEF8BDC82920001C6810001FF021E323
:206820000400A0E10040BDE81EFF2FE1F0009FE5003090E5F84F2DE9E8009FE5001090E55A
:2068400004D081E513F021E3DCD09FE5DC009FE50FE0A0E110FF2FE19FF021E3C4009FE5FD
:20686000001090E504D091E5F84FBDE8B0009FE5003080E51EFF2FE100402DE9B0009FE5DD
:206880000FE0A0E110FF2FE10040BDE8A4009FE590109FE5001091E5000051E398109F0532
:2068A0001320A0030600000A001090E5182010E59FF021E306002DE993F021E37C109FE5FA
:2068C0001F20A0E3001080E5182000E51EFF2FE10F502DE9D4FFFFEB64009FE50FE0A0E1AD
:2068E00010FF2FE118208DE292F021E30300B2E801F06FE100E0A0E19FF021E30F50BDE876
:2069000008D08DE292F021E304F05EE2F05F2DE90D00A0E193F021E300D0A0E1F05FBDE8B7
:206920001EFF2FE1C8292000D0292000983F20008566100075641000D43F20004C6810002E
:20694000D46810006964100070470000704700007047000000B50C480068C00712D50B4877
:206960000068FFF7B5F8FEF75BF84B480168491C016007480068081A04D45C480178012211
:206980000A43027000BDC04634FDFFFF38FDFFFF6800200030B51F481F4901601F482049A6
:2069A00008609F21C9431F4A0A601F491F4A0A601F490A68D207FCD51E4A1F4B13600A685A
:2069C0005207FCD508220B681342FBD01B4B07241C6008240B682342FCD00021C943184B63
:2069E0001960184B19604949174B0B601749184B0B600121454C174D8B00E550491C202930
:206A0000FADB394900230B60521EFAD112490860012030BD44FDFFFF0062FF0F010000A530
:206A200040FDFFFF0001480020FCFFFF0106000068FCFFFF2CFCFFFF051C191030FCFFFFB5
:206A400024F1FFFF28F1FFFF4969100034F1FFFF516910004D69100008FDFFFF00B5FFF7E9
:206A6000EDFC0648064901600649012000F040F8012000F04DF8FFF747FD00BD30FDFFFF1F
:206A8000B20B00035569100000B5024801210160FDE7C04604FCFFFFC429200010B51048D4
:206AA0000068104C2178491C21706178491C617000F0A8FE0C48002101606078401E607002
:206AC0002078012805D109480078002801D000F04BF82078401E207010BC01BC0047C046CE
:206AE00000F1FFFFC829200030F1FFFF0434200030B505000C00FFF7A1FCA8000349081882
:206B000005680460FFF700FD280030BD80F0FFFF10B50400FFF792FC03480121A140FFE7AD
:206B20000160FFF7F1FC10BD20F1FFFF10B50100054A137818008B4205D00121FF24E4436F
:206B400021605940117010BD053420000020EDE700B5402281214903D00300F01DFE01207C
:206B6000FFF7E4FF00BD0000004B18477868100010B52A4CE068002806D0FFF7C3F8E0686B
:206B8000FFF736FB0020E060002010BDF7B504000025224EF068002805D1FFF7EBFB0020EA
:206BA000FFF7E8FBFEBD02A901A8FFF7B5F801983169471A05D10298002805D17769012542
:206BC00002E001D570693F18A74200D23C002800FFF7D0FB2000FFF7CDFB002C10D030696A
:206BE000019988420ED3F168091A72698F18A74200D327003900FFF78BFBE41BF0683061D2
:206C0000002C06D021003069FFF782FB3069001930613069FFF788F8FEBD00006C002000AC
:206C200011B504E068460178201DFFF7C1FB01216846FFF7BDFB2B4C68460078002835D14B
:206C40006068FFF79BF802001068516800F014FEA068814200D2A1601068916800F00CFEA5
:206C6000A068884200D2A160E068002807D06169226891420CD0FFF7BBFA0020E060206892
:206C8000FFF792FAE06020686061E068002809D0FFF738F82368E268A1686068FEF7F2FFEE
:206CA000E06820610020FFF765FB18BD012100A8401CFFF77DFB684640780128B2D00228F1
:206CC00002D0042805D008E06846017808342000ABE7684601782000A7E7684601780020C8
:206CE000A3E7C0466C00200003B5012100A8801CFFF75EFB002069468978642932D065291E
:206D00003DD0662948D06E292BD1019002E001A8FFF74EFB01216846FFF74AFB68460078A0
:206D2000002805D1019800280FD00020C04330E0012100A8401CFFF73BFB684640780128A1
:206D400068460178E3D00020E2E71C20FFF712FB0198FFF70FFB0198FFF710F81421FFF7D6
:206D6000D7FA0CBDFFF75CFF0CBD012100A8401CFFF71EFB684601780020FFF719FB0121B7
:206D80006846FFF715FB684600780028EDD1FFF7EFFEFFF7EFFA0CBD019002E001A8FFF796
:206DA00007FB01216846FFF703FB68460078002803D10198FFF7EAFE0CBD012100A8401C85
:206DC000FFF7F6FA68464078032868460178E5D00020E4E7CCE60000D2F021E30CD09FE59D
:206DE000DFF021E308D09FE508009FE510FF2FE1D83F2000983F2000FC20100000B5FFF7B4
:206E000015F900BD00B5FFF7FBF84007400F00BD3FB5010002A8154A13680360536843607C
:206E20000A06120E900842401206120E012368468C08012525406C008907C90E214354084C
:206E400062401C00544023405A010A4385211143017005220021401C00F0FCFC6A4602A983
:206E60002E20FFF703F9083004B030BD748610007FB50C0002A91A4A13680B6053684B6054
:206E80000106090E8A0851400906090E01226D46830801261E4073008007C00E18434B082F
:206EA00059400A405101014381200843287000206870687105222100681CFCF0D3FE20005B
:206EC000FCF07AFF00066979C00C084368716A4602A93020FFF7CAF8083004B070BDC046F3
:206EE0007C86100001480078704700000734200000B500F0CDFB00F0E9FB00BDF0B5040006
:206F00000D00744E7068401B7060B068311880229200131A9D4208D22A001831200000F0A1
:206F200015FBB0684019B060F0BD171A3A001831200000F00BFBED1B2A0031001831E019A4
:206F400000F004FBB560F0BD00B500F0A3FA61494869002804D0486900224A6100F004F87D
:206F600000F08AFA00BD0000F0B504008027BF00584DE86800281AD0EE68B44200DA26007E
:206F8000002231002869FCF085FD286980192861A41BE868801BE860E868002810D1287801
:206FA00000280DD00020287000F082FA08E06868381AA04203D26C6100F060FBF0BD0026FC
:206FC000002C30D03604360C6868002809D13200210028001830FCF05DFD6C600020A8603A
:206FE00021E0391AA1421ED3A9680818B84201D30F4940183F1AA74200DB2700320039000B
:2070000028181830FCF046FDE41B6868C0196860002C08D0F219210028001830FCF03AFD86
:2070200068680019686000F073FA00F029FBF0BD00FEFFFFF0B505000E00FFF753FF00285D
:2070400000D1F0BD34000DE0FE603D61FFF77CFFF868002803D00120387000F02DFAFE6883
:2070600000F00EFA002E10D000F018FA194F78680028E9D03700874200DB0700390028009C
:20708000FFF73CFFF61BED19EAE72000F0BD0000F0B506000D00FFF725FF002818D000F038
:2070A000FDF90C4C002D0BD06768002F0AD0BD4200DA2F0039003000FFF720FFED1BF61905
:2070C000002D03D0E5602661FFF73EFF00F0D8F9F0BD0000B0002000014800687047C04605
:2070E000BC00200030B504000D00A078E178014303D1A079E179014302D000F031FA30BDA4
:207100008D4800780028F8D0FFF7ECFE0028F4D020788007800F02D0022806D0EDE70122EF
:207120000021002000F052FA30BD844821790029F5D0022909D08129DFD10178FE220A4050
:207140000121294011430170E9E70178FD220A40690002230B4013430370E0E7F3B5060016
:2071600000F08AFA31786020084015D130790190B0786A4F704D002472780B2A12D802A39A
:207180009B5C5B009F44C04606447D467D4B5B7D8D95ACBDF278024373D1B079F2790243B0
:2071A000022A00D06DE0287800286AD003220A4000A8801C397800290AD1012A02D9921E66
:2071C00002D0FCBD04701DE001990029FAD058E0002A04D0012AF5D0022A02D012E00121EE
:2071E0000FE05649019A002AECD0022A06D0812A47D1097801220A40027003E009780A40AD
:207200005108017044700022022100A8801C45E0002100E001213000FFF764FFFCBD0600D7
:2072200001220021080000F0D1F9300000F09EF9002E00D001242C7000F090F9FCBD00257B
:2072400000F018FAF078012804D0022804D0032805D014E0324D12E0324DAC780FE0B078AA
:2072600003280CD801A1095C8F44C04604080C102D4D04E02D4D02E02D4D00E02D4D002D3C
:2072800002D100F06DF9FCBD002C00D12C78B079A04200DA040001222100280000F096F997
:2072A000FCBDFFF71FFE69460870002201216846F4E700F053F9B078012809D10122002163
:2072C000080000F083F90120387000F05DF9FCBD0028D6D10122002100F078F93C70FCBD99
:2072E0000028CED1B079012800D0CAE728780028C7D038780028C4D06846047000220121C3
:20730000CCE7019829780029BBD03978002900D1B7E70006000E0228B3E7C046073420004A
:207320008400200084861000A4861000A8861000B88610009800200008342000063420005B
:2073400030B504000D0000F0A9F801E000F0C6F800F000F90028F9D029002000FCF058FBB5
:2073600000F08EF830BD000030B5424C6568002D0DD0412D00DB402529002068FFF7E0FF2C
:207380006068401B606020684019206030BD00F099F830BD00210020D2E7000030B504006B
:2073A0000D0000F07BF809480068002801D000F095F800F065F805E040212000FFF7C0FFC6
:2073C0004034403D402DF7D202E0C046E429200029002000FFF7B4FF30BD0000F1B50E00DE
:2073E000FFF72CF8224C6078401C6070214D6968002918D0401E2A685218009B9A4204D10B
:20740000891969606070002823E06070002801D1FFF70AF800F09EF80028FBD0FFF70EF8CF
:207420006078401C607000F095F8002815D03700412F00DB402739000098FFF781FFF61B7D
:207440000098C0190090002EEDD16078401E607000060CD1FEF7E8FFF8BD009828606E60D7
:207460006078401E6070000601D1FEF7DDFFF8BDC8292000E029200000B5FFF745F800BDC9
:2074800000B50A484178491E4170090601D1FEF7CBFF00BD00B5FEF7D1FF00BD00B5FEF7D6
:2074A000CDFF02484178491C417000BDC829200010B5034C08E0000000B5014810E000002F
:2074C000E829200010B50A4C2168002904D00120FEF7D8FF0020206010BD000000B504487F
:2074E0000449096801600120FEF7EAFF00BD0000EC292000D029200000B504490B20FFF740
:20750000F7FA0B20FFF704FB00BDC046F93A200010B50C4901222A48036842241C40402CFC
:2075200000D10A600B685A400A60016803D0022291434F4A02E040229143034A0A430260B8
:2075400010BDC046F02920000F80000000B500F023F900BD1C4800687047000070470000D8
:2075600042480168004A09E06F80000005498022520002430A601348016801220A4302606F
:207580007047C0460800FBFF0C48C021C90001600B49802292000A60920103681343036024
:2075A000086802430A60022006490A6802430A60364906220A600449086070473400FBFF6F
:2075C0003800FBFF0400FBFFF4292000F4B50122D243264B1C681440214D25431D6004E0DD
:2075E00015401F4E2E431E60091B0906090E1CD00025082903D26C4625700C0008E009290C
:20760000FBD3082404E0174E07783760401C6D1CA542F8D31D68144E2E431E601D68ED072B
:207620001D68DDD4AD07F9D50DE068460078002814D018680C49014319601868C00718681A
:2076400008D48007F9D5186802218843084901431960F8BD0240024810431860F8BDC046B6
:207660004E8000005000FBFF5F8000003000FBFF4D8000007047000070470000124801E073
:207680000248C04604210160704700001000FBFF00B5FFF7FFFEFFF72FFF08488021016035
:2076A00007480901016008480021C9430160054800210160FFF7E0FE00BDC04600FCFFFFD2
:2076C00010FCFFFF7400FBFF1400FBFF802040050349086003490860034908607047C04666
:2076E00000F4FFFF10F4FFFF30F4FFFF0102000A08430004000C7047F6B504001D00072161
:207700000A4209D1D60832000099200000F044F8A4196D1EF7D1FCBD0020009A019901E050
:20772000641C08391378521C00280AD083402678FF278740BE431F00374327701B0A637016
:2077400000E023700829EBDA4018C10864184007400F6D1EE1D1FCBD00B5884200DB080035
:2077600000BD000002681170521C02607047000002681170090A5170921C02607047000054
:2077800002681170090A5170090A9170090AD170121D026070470000004B1847A0342000DC
:2077A00010B5FDF709FFFEF711FB0020FEF72CFBFEF744FE0C484178491C4170FBF03EFF49
:2077C000FFF7C6F9FEF7CEFFFFF748F90748084902B40300074A6421054C0019FEF7FAFF74
:2077E00000F00AF818BDC046C8292000802A20006809000055621000004B18474468100043
:2078000000B5FEE70047000000B581B000F02EF801B000BD10B5002A0DD003780C78A3426D
:2078200005D002D20020C04310BD012010BD401C491C521EF1D1002010BD000010B5030019
:20784000002A05D00C78491C1C705B1C521EF9D110BD000000B50906090E0300002A03D05B
:2078600019705B1C521EFBD100BD0000014CA64620470000017810007847C0460C002DE9FF
:2078800000C0A0E3060000EA7847C0460C002DE941C0B0E1001061228CC0A0E140C03CE0C0
:2078A000000060220120B0E13100000A0030A0E3200851E10118A091200451E10114A09166
:2078C000A00051E12000008A200151E11C00008AA00151E11700008A200251E11200008ACF
:2078E000A00251E10D00008A200351E10800008AA00351E10300008A810350E1810340203B
:207900000330A3E0010350E1010340200330A3E0810250E1810240200330A3E0010250E1E1
:20792000010240200330A3E0810150E1810140200330A3E0010150E1010140200330A3E098
:20794000810050E1810040200330A3E0010050E1010040200330A3E0020051E12114A0810B
:20796000E4FFFF8A0310A0E18C3FB0E100106122000060420C00BDE81EFF2FE17847C046D3
:20798000F0412DE90140A0E10280A0E10350A0E1006090E570709FE52200D7E5000050E3BD
:2079A0000C00000A040094E4FC0100EBA86186E0078008E20820A0E10010A0E10600A0E1AC
:2079C000040200EB880097E5088080E0015055E2F3FFFF1A090000EA041094E4A86186E049
:2079E000078008E20820A0E10600A0E1F90100EB880097E5088080E0015055E2F5FFFF1A80
:207A00000400A0E1F041BDE81EFF2FE1DC022000030052E33D00009A03C010E20800000A0A
:207A20000130D1E402005CE30C2082E001C0D1940130C0E40130D13401C0C094042042E203
:207A40000130C034033011E21D00000A042052E22E00003A03C031E7020053E30800000ACF
:207A60000F00008A2C34A0E104C0B1E5042052E20C3C83E1043080E4F9FFFF2A011081E201
:207A8000220000EA2C38A0E104C0B1E5042052E20C3883E1043080E4F9FFFF2A021081E26D
:207AA0001A0000EA2C3CA0E104C0B1E5042052E20C3483E1043080E4F9FFFF2A031081E254
:207AC000120000EA202052E210402DE90500003A1850B1E81850A0E81850B1E81850A0E8AF
:207AE000202052E2F9FFFF2A02CEB0E11850B1281850A0281800B1481800A04802CFB0E1AC
:207B00001040BDE804309124043080241EFF2F01822FB0E10120D1440130D12401C0D1240E
:207B20000120C0440130C02401C0C0241EFF2FE1F1B504000D001600174800681F2188439A
:207B40008027202100911549884202D01449884202D180374020009000F038F82000009938
:207B60002A6822602D1D241D491EF9D1802F00D140009B21C9430B4A02400B481043086008
:207B80009720C0430068C007FAD5F61B012EE5DA02F772FFF8BDC04640F2FFFF40090D275C
:207BA00040095B2700FF03000100005A00B59720C0430168C90606D49B21C943024A0A609E
:207BC0000168C907FCD500BD0F00005A004B1847406410007847C046F0072DE91CC09DE5E7
:207BE00020409DE5EF50E0E3C05FC5E3496FA0E3006085E5FB50E0E3B05EC5E3706AA0E3B4
:207C0000006085E58060A0E3006082E5B4609FE5307096E5047082E5346096E5306082E5DC
:207C20000160A0E3006082E5807CA0E3007083E5046083E50770A0E31C7083E50280A0E383
:207C4000188083E5408FA0E3008083E50180D0E4248083E58088A0E30C9085E2008089E52D
:207C6000309085E3008089E52CA085E200808AE5008089E500808AE5008089E500808AE512
:207C8000109085E3008089E52180A0E3108083E5147083E5006083E5606CA0E3006085E505
:207CA000081182E5080183E500C183E5010044E20C0183E5044183E5FA0087E2200183E575
:207CC000F007BDE81EFF2FE15804200006214843401EFDD170470000F04F2DE9FF70E0E343
:207CE000B07EC7E340BCA0E303E0A0E10140D0E40150D1E480CBA0E30880A0E3080053E3B7
:207D00000380A041083043E000A0A0E3A440B0E180AB8A23A550B0E180AD8A2338A087E590
:207D200001C05CE21900000A3CA097E540001AE3FAFFFF1A30B087E501C05CE21300000A12
:207D40003CA097E540001AE3FAFFFF0AAAA6B0E16660A0E1018058E2EAFFFF1A266CB0E184
:207D60000160C2E4000053E3DFFFFF1A07301EE2083063123663A011016042150000A0E366
:207D800080ADA0E334A087E5F04FBDE81EFF2FE130B087E50100A0E3F8FFFFEA224B184766
:207DA000224B1847F0B5FFF7F9FF214F0024402501263603BC63C046F86BF96BFA6BFB6B54
:207DC000FC6B2C4204D0761EFAD10020401E10E0284220D0294220D02A4220D02B4220D0BF
:207DE00001210903881B0921484315214843C830733040242402BC6301263603761E07D02D
:207E0000FC6B2C42FAD0041CFFF7CAFF201CF0BD0020401EF7E70020EBE77E20E9E7BD2062
:207E2000E7E7FC20E5E70000406410002C64100000F4FFFFF04F2DE924409DE5FF90E0E3B9
:207E4000B09EC9E310A0A0E380B6A0E303E0A0E1000054E32200000A0150D0E40160D1E45A
:207E60000880A0E3080053E30380A041083043E0A550B0E110A0892514A08935A660B0E10D
:207E800030A0892534A0893530B089E504C0A0E101C05CE2FDFFFF1A34B089E504C0A0E194
:207EA00001C05CE2FDFFFF1A3CC099E5ACC2B0E16770A0E1018058E2ECFFFF1A277CB0E1EA
:207EC0000170C2E4000053E3E2FFFF1A07301EE2083063123773A01101704215F04FBDE870
:207EE0001EFF2FE10150D0E40160D1E40880A0E3080053E30380A041083043E0A550B0E1AC
:207F000010A0892514A08935A660B0E130A0892534A0893530B089E534B089E53CC099E5D0
:207F2000ACC2B0E16770A0E1018058E2F2FFFF1A277CB0E10170C2E4000053E3E8FFFF1AA4
:207F4000E1FFFFEA0F502DE900004FE101002DE993F021E300402DE91C009FE50FE0A0E1AF
:207F600010FF2FE10040BDE892F021E30200BDE801F06FE10F50BDE804F05EE29D6A100040
:207F800000B51F4A102923D3037813604378136083781360C378136003791360437913603E
:207FA00083791360C3791360037A1360437A1360837A1360C37A1360037B1360437B136041
:207FC000837B1360C37B1360103010391029DBD2002904D003781360401C491EF8E703F789
:207FE00011FD6B484168491E4160012904D169480168694A0A43026003F7F6FC00BDC046E5
:208000005400FBFF00B5174A102923D31368037013684370136883701368C37013680371A6
:2080200013684371136883711368C3711368037213684372136883721368C37213680373C2
:2080400013684373136883731368C373103010391029DBD2002904D013680370401C491EB0
:20806000F8E700BD5800FBFFF3B53A4804683A480068044039480460454DA00713D54548BB
:20808000016801229143364A0A4302606968022909DA491C6960022905DA01683E4A0A43FC
:2080A000026003F719FC04210C4205D02D4800684001400D03F710FA2B48044249D00026A0
:2080C0002A4FE00724D53868042108421ED000216846274A12684254491C0829F9DB3968EF
:2080E00004229143234A0A433A600078000603D53868214901433960684603F7E7FA3868CC
:20810000802188431D490143396001E048033860E00410D51A480021C9430160066019486C
:208120008021490001603868C901014339602E6015480121016020070BD53868202188438C
:208140000E49014339603868082188430F4901433960FCBD1800FBFF1C00FBFF2000FBFF27
:208160004E8000003800FBFF091000003000FBFF5000FBFF4B800000CF8000004F80000089
:208180002800FBFF0800FBFF1000FBFF47800000F02920003400FBFF5F8000007847C046DF
:2081A00028109FE5202CD1E70034A0E1233CD1E7032482E10038A0E1233CD1E7032882E14B
:2081C000000CA0E1200CD1E7000C82E11EFF2FE1C88610007847C046033000E2832182E054
:2081E0000300C0E3000052E30A00000A0130A0E31332A0E1013043E200C090E50CC003E0DC
:2082000011C28CE104C080E400C090E50330CCE1202062E2311283E1001080E51EFF2FE114
:208220007847C04630002DE900C0A0E3A10180E0071011E20900000A084041E2033084E0CF
:2082400001C0D2E40040D0E5FF50A0E31551E0E1044005E01C51A0E1044085E10140C0E413
:20826000081061E2080053E32200003AA341A0E1140000EA0150D2E405C48CE13C51A0E15B
:208280000150C0E40150D2E40554A0E12CC485E13C51A0E10150C0E40150D2E40554A0E1CE
:2082A0002CC485E13C51A0E10150C0E40150D2E40554A0E12CC485E13C51A0E10150C0E42B
:2082C0002CC4A0E1044044E2040054E3E8FFFF2A000054E30600000A0150D2E405C48CE1F4
:2082E0003C51A0E10150C0E42CC4A0E1014044E2F6FFFFEA073003E2000053E30700000A62
:208300000020D2E502248CE13211A0E10120A0E31223A0E1012042E2011002E00010C0E5E8
:208320003000BDE81EFF2FE17847C046200820E0200420E0200220E0200120E0A00020E047
:20834000010000E21EFF2FE142310000C8022000C8022000CC0900000C3420007C7910008C
:20836000880200004000200078831000CC0900000C3420007C7910000000000001000000CD
:208380000400000000000000000000000000000000000000000000000000000000000000D9
:2083A0000040000000100000000000008025000000000000000000000000000012011001A4
:2083C000000000086613010101000102030100000E0331003200330034003500360030009C
:2083E0003000300030000000010000000000000000000000000000000000000000000000EC
:2084000000000000000000000000000000000000000000000000000000000000000000005C
:2084200000000000000000000000000000000000000000000000000000000000000000003C
:2084400000000000000000000000000000000000000000000000000000000000000000001C
:208460000000000000000000000000000000000000000000000000000000000000000000FC
:208480000000000000000000000000000000000000000000000000000000000000000000DC
:2084A0000000000000000000000000000000000000000000000000000000000000000000BC
:2084C00000000000000000000000000000000000000000000000000000000000000000009C
:2084E00000000000000000000000000000000000000000000000000000000000000000007C
:2085000000000000000000000000000000000000000000000000000000000000000000005B
:2085200000000000000000000000000000000000000000000000000000000000000000003B
:2085400000000000000000000000000000000000000000000000000000000000000000001B
:208560000000000000000000000000000000000000000000000000000000000000000000FB
:208580000000000000000000000000000000000000000000000000000000000000000000DB
:2085A0000000000000000000000000000000000000000000000000000000000000000000BB
:2085C00000000000000000000000000000000000000000000000000000000000000000009B
:2085E00000000000000000000000000000000000000000000000000000000000000000007B
:208600004941524B53000000BF7BFF194A616E4665624D61724170724D61794A756E4A7512
:208620006C4175675365704F63744E6F76446563701101007011010070110100701101001C
:2086400070110100701101007011010070110100808D5B0001000000FFFF000000000000AB
:2086600000000000B1631000156410002164100011631000FF00000000E00000FFE0FFFF78
:20868000FFFF000009022000010100C0320904000002FFFFFF0007058102400000070502D4
:2086A00002400000040309040E0353004500470047004500520000000E034A002D004C00C2
:2086C00069006E006B000000008040C020A060E0109050D030B070F0088848C828A868E818
:2086E000189858D838B878F8048444C424A464E4149454D434B474F40C8C4CCC2CAC6CEC9A
:208700001C9C5CDC3CBC7CFC028242C222A262E2129252D232B272F20A8A4ACA2AAA6AEA89
:208720001A9A5ADA3ABA7AFA068646C626A666E6169656D636B676F60E8E4ECE2EAE6EEE19
:208740001E9E5EDE3EBE7EFE018141C121A161E1119151D131B171F1098949C929A969E951
:20876000199959D939B979F9058545C525A565E5159555D535B575F50D8D4DCD2DAD6DEDF9
:208780001D9D5DDD3DBD7DFD038343C323A363E3139353D333B373F30B8B4BCB2BAB6BEBE9
:2087A0001B9B5BDB3BBB7BFB078747C727A767E7179757D737B777F70F8F4FCF2FAF6FEF79
:2087C0001F9F5FDF3FBF7FFFFF8F4FCF2FAF6FEF0000000000000000000000000000000039
:2087E000000000000000000000000000000000000000000000000000000000000000000079
:20880000000000000000000000000000000000000000000000000000000000000000000058
:20882000000000000000000000000000000000000000000000000000000000000000000038
:20884000000000000000000000000000000000000000000000000000000000000000000018
:20FF0000FFFFFFFF000000000000000000000000FFFFFFFFFFFFFFFFFFFFFFFFFFFFFFFFF5
:020000040010EA
:20FF200052444900FFFFFFFFFFFFFFFFFFFFFFFF466C617368425000FFFFFFFFFFFFFFFF76
:020000040010EA
:20FF4000466C617368444C00FFFFFFFFFFFFFFFF4A466C61736800FFFFFFFFFFFFFFFFFFFC
:020000040010EA
:20FF600047444246756C6C00FFFFFFFFFFFFFFFFFFFFFFFFFFFFFFFFFFFFFFFFFFFFFFFF39
:020000040010EA
:20FF8000FFFFFFFFFFFFFFFFFFFFFFFFFFFFFFFFFFFFFFFFFFFFFFFFFFFFFFFFFFFFFFFF81
:020000040010EA
:20FFA000FFFFFFFFFFFFFFFFFFFFFFFFFFFFFFFFFFFFFFFFFFFFFFFFFFFFFFFFFFFFFFFF61
:020000040010EA
:20FFC000FFFFFFFFFFFFFFFFFFFFFFFFFFFFFFFFFFFFFFFFFFFFFFFFFFFFFFFFFFFFFFFF41
:020000040010EA
:20FFE000FFFFFFFFFFFFFFFFFFFFFFFFFFFFFFFFFFFFFFFFFFFFFFFFFFFFFFFFFFFFFFFF21
:00000001FF
